:020000040000FA
:020000003529A0
:08000800AA00030E8301AB0006
:100010000408A9008C1A15280B1935282908840012
:100020002B0E8300AA0E2A0E090098182D281819E5
:100030002D281A08A30025082402031920282228A5
:10004000A501A401A40A2408A03E84002308831665
:1000500003138000831203130A281A081A081A08C7
:10006000181218161A081A080A280B117330810082
:10007000281C0A280C3026020319492804302602BD
:10008000031C4C28A70C03180614031C0610A60317
:100090000A280610A6030A280614A6030319281026
:0200A0000A282C
:06026A0000308501860151
:100270008A0107309F0083168F308100003085008F
:100280001230860020309900181518128312981722
:1002900020308B00831620308C00831200308C00BD
:1002A000A401A501A801A60183160B118B168312C8
:1002B000181218168B171F3085000130860025088C
:1002C000240203195F2928185F290C30A60025088D
:1002D000013EA03E8400831603130008831203131B
:0802E000A700A50A28145F29FC
:02400E00A23FCF
:00000001FF
